:0400000002EF1AF001
:1000080000C015F0E1CF16F0E2CF17F09EAA4ED04F
:100018009DAA4CD0AFCF60F0ACA202D0AC98AC880F
:10002800ACA404D0AFCF60F03F0EAE6E00016051BB
:100038000D0A14E19D9A010E746F000E756FCA0EB9
:100048009D25E16E000E9E21E26EE66A9DC061F07C
:100058009EC062F09D6B9E6B606B0ED0CA0E9D2594
:10006800E16E000E9E21E26E60C0E6FF9DC061F069
:100078009EC062F09D4B9E2B000E9E5D02E1800E9D
:100088009D5D13E3020E746F000E756F9D9ACA0E84
:100098009D25E16E000E9E21E26EE66A9DC061F02C
:1000A8009EC062F09D6B9E6B606BACD7A4AA4DD0CE
:1000B800A3AA4BD09CA202D09C989C889CA402D056
:1000C800AACFC9F00001AACFC9F0C9510A0A12E1A2
:1000D800010E6D6F000E6E6F5B0E2E24E16E020E28
:1000E8002F20E26EC9C0E6FF2EC021F02FC022F0FB
:1000F800C96B0ED05B0E2E24E16E020E2F20E26E2D
:10010800C9C0E6FF2EC021F02FC022F02E4A2F2AA8
:10011800010E2F5C02E1000E2E5C17E3020E6D6FDC
:10012800000E6E6FA39A010E2E5E000E2F5A5B0E04
:100138002E24E16E020E2F20E26EE66A2EC021F018
:100148002FC022F02E6A2F6AC96BF2AA1AD0F2A425
:1001580018D00301CD4BCE2B000E006ECE51005CA3
:1001680002E1CD51090808E2010ECF6F000ED06FF1
:10017800F29ACD6BCE6BD59E480ED76EE50ED66E35
:10018800F2949DA01BD09EA019D00101CD4BCE2B7F
:10019800000E006ECE51005C02E1CD51640804E20D
:1001A800240EAE6ECD6BCE6B010ECB6F000ECC6FF6
:1001B800CD906D0ECF6E840ECE6E9E9015C000F061
:0A01C80016C0E1FF17C0E2FF1100AE
:1001D2000B820BAEF3EF00F003680268016800685F
:0801E2000A360232FF0E120082
:0E01EA00026A016A006A086A036A000E1200C7
:1001F8000B840BAE07EF01F0010E036E026A016A71
:0A020800006A0A360232FF0E1200EF
:080212000AAE029E000E12006C
:10021A00C7B409D01F0EC514016E0150000A03E1CC
:0A022A00010E006E01D0006A120000
:100234000CB05CEF01F00CA202EF02F00E6A000EAB
:10024400026473EF01F0F00E0214D8A43EEF01F043
:10025400023A01380F0B02260138F00B016E003808
:100264000F0B01260038F00B006E08380F0B002628
:100274000838F00B086E0E84D89002BE57EF01F0D8
:1002840008360036013602360E2A02BE57EF01F058
:1002940008360036013602360E2A02BE57EF01F048
:1002A40008360036013602360E2A0E500364F8EF83
:1002B40001F0035E0BBC08AEFDEF01F0D880800EA8
:1002C40008640030000E002201220222D8A0FDEFB3
:1002D40001F0023201320032034A02EF02F0FDEF74
:1002E40001F001C002F000C001F008C000F0086A8B
:1002F400000E0E860264AAEF01F0F00E0214D8A4D8
:1003040092EF01F0023A01380F0B02260138F00B8C
:10031400016E00380F0B01260038F00B006E0E84BE
:10032400D89002BE57EF01F00036013602360E2A8D
:1003340002BE57EF01F00036013602360E2A02BE25
:1003440057EF01F00036013602360E2A57EF01F05E
:1003540001C002F000C001F0006A000E0E960E8883
:100364000264D7EF01F0F00E0214D8A4C2EF01F03A
:10037400023A01380F0B02260138F00B016E0E848D
:10038400D89002BE57EF01F0013602360E2A02BEA3
:1003940057EF01F0013602360E2A02BE57EF01F084
:1003A400013602360E2A57EF01F001C002F0016A4D
:1003B400000E0E86026407EF02F0F00E0214D8A4B9
:1003C400E6EF01F0023A0E84D89002BE57EF01F036
:1003D40002360E2A02BE57EF01F002360E2A02BE82
:1003E40057EF01F002360E2A57EF01F0010E0C6EA2
:1003F40001DF0AEF02F0020E0C6E09DF0AEF02F0D1
:10040400040E0C6EE4DE0AEF02F0080E0C6EEBDE56
:020414001200D4
:100416000B800BAE17EF02F0026A0AAEFF0E026EF9
:0C042600016E006E0A360232FF0E12005A
:0A043200C582C5A201D0FDD712005B
:0E043C00570E0D6E0D2EFED7000000001200B0
:10044A00086A096A100E0C6E01340836093604501F
:10045A00085E0550D8A0053C095ED8B007D0045004
:10046A0008260550D8B0053C0926D8900036013632
:06047A000C2EEAD712006F
:100480009E9640C4C9FFC7A401D0FDD79EB601D037
:10049000FDD7C5BC02D0006A03D0C584020E006E31
:0204A000120048
:1004A2000C6A0E6A0250D8A46AEF02F001C002F090
:1004B20000C001F0006A0E860250D8A46AEF02F072
:1004C20001C002F0016A0E960E880250D8B47CEF89
:1004D20002F00E50035ED8A4D8A081EF02F0D890AB
:1004E20002BE86EF02F0003601360236032E71EFAD
:1004F20002F081EF02F0010E0C6E76DE89EF02F05F
:10050200020E0C6E78DE89EF02F0040E0C6E80DEB5
:020512001200D5
:100514000401406B416B4151120802E140518E08C5
:1005240008E379DE005201E004D00401404B412B82
:10053400F2D70401120E415D02E18F0E405D03E328
:100544007B0E006E05D0C580C5A001D0FDD7006A22
:02055400120093
:080556000B6A0B86FF0E120078
:10055E0042C4F6FF43C4F7FF44C4F8FF0900F5CFC9
:10056E0000F0005218E042C4F6FF43C4F7FF44C443
:10057E00F8FF0900F5CF00F040C4E1FF41C4E2FFEF
:10058E0000C0E6FF0401404B412B010E4227000E36
:10059E0043234423DDD740C4E1FF41C4E2FFE66AB2
:0205AE00120039
:1005B000025006180E6E086A096A0B6A0350076437
:1005C000CBEF03F006500A6E068E028E03500B6EC0
:1005D0000750036E000E0B641BEF03F00B50075E19
:1005E000D8B4BCEF03F0070E07648AEF03F0075E90
:1005F00000C008F001C000F002C001F0026A074E1E
:10060000BCEF03F007645FEF03F0075E00C008F083
:1006100001C000F0016A074EBCEF03F007643DEF34
:1006200003F0075E00C008F0006A074EBCEF03F05D
:10063000076424EF03F00AC002F005C001F004C013
:1006400000F0086AE5EF04F0030E07642FEF03F0F3
:10065000075E08380F0B086E074EBCEF03F0D8900A
:100660000832074EBCEF03F0D8900832074EBCEFBB
:1006700003F0D8900832BCEF03F0030E07644EEF8E
:1006800003F0075E08380F0B086E0038F00B0826E1
:1006900000380F0B006E074EBCEF03F0D89000320D
:1006A0000832074EBCEF03F0D89000320832074EF4
:1006B000BCEF03F0D89000320832BCEF03F0030E19
:1006C000076476EF03F0075E08380F0B086E0038FA
:1006D000F00B082600380F0B006E0138F00B0026D7
:1006E00001380F0B016E074EBCEF03F0D8900132BA
:1006F00000320832074EBCEF03F0D89001320032CE
:100700000832074EBCEF03F0D890013200320832B5
:10071000BCEF03F0030E0764A7EF03F0075E083891
:100720000F0B086E0038F00B082600380F0B006E18
:100730000138F00B002601380F0B016E0238F00B68
:10074000012602380F0B026E074EBCEF03F0D89063
:100750000232013200320832074EBCEF03F0D8906B
:100760000232013200320832074EBCEF03F0D8905B
:100770000232013200320832096A000E0EAEB0EFCA
:1007800004F0081E001E011E021E082A002201227B
:100790000222B0EF04F00750D8A4D1EF03F0E5EF48
:1007A00004F0096A02C00AF0028E068E0750035C4C
:1007B000076ED8B4A3EF04F0070E076471EF04F0DE
:1007C000075E0450096E0550046E0650056E066AF9
:1007D000074EA3EF04F0070E076446EF04F0075E30
:1007E0000450096E0550046E056A074EA3EF04F02D
:1007F000070E076424EF04F0075E0450096E046AD4
:10080000074EA3EF04F0070E07640BEF04F00AC0D5
:1008100002F0E5EF04F0030E076416EF04F0075E44
:1008200009380F0B096E074EA3EF04F0D890093278
:10083000074EA3EF04F0D8900932074EA3EF04F05F
:10084000D8900932A3EF04F0030E076435EF04F0EB
:10085000075E09380F0B096E0438F00B09260438BF
:100860000F0B046E074EA3EF04F0D8900432093248
:10087000074EA3EF04F0D89004320932074EA3EFDD
:1008800004F0D89004320932A3EF04F0030E076499
:100890005DEF04F0075E09380F0B096E0438F00BAA
:1008A000092604380F0B046E0538F00B04260538B2
:1008B0000F0B056E074EA3EF04F0D89005320432FB
:1008C0000932074EA3EF04F0D89005320432093202
:1008D000074EA3EF04F0D890053204320932A3EF9B
:1008E00004F0030E07648EEF04F0075E09380F0B67
:1008F000096E0438F00B092604380F0B046E053816
:10090000F00B042605380F0B056E0638F00B052694
:1009100006380F0B066E074EA3EF04F0D890063290
:10092000053204320932074EA3EF04F0D8900632A4
:10093000053204320932074EA3EF04F0D890063294
:10094000053204320932086A000E0EAEB0EF04F030
:10095000091E041E051E061E092A0422052206225F
:100960000950082604500022055001220650022298
:100970000EBEC7EF04F0D8A0D6EF04F00232013269
:1009800000320832033ED6EF04F0E0EF04F0D8B0B6
:10099000DBEF04F0000E081E001E011E021E082AD6
:1009A0000022012202220A7EDBEF04F0010E0C6E0F
:1009B00041DCE7EF04F0020E0C6E3CDCE7EF04F0E4
:1009C000040E0C6E06DCE7EF04F0000E0C6E120055
:1009D00040C402F041C403F002C000F003C001F0C3
:1009E000024A032A00C0E9FF01C0EAFFEE5201E01B
:1009F000F3D704014051025C006E41510358016E6F
:0A0A0000010E005E000E015A120004
:100A0A0044C400F004014407005228E040C4E9FF4E
:100A1A0041C4EAFFEE50000A0CE040C4E9FF41C4B9
:100A2A00EAFF42C4D9FF43C4DAFFEE50DE1801E1FF
:100A3A000FD040C4E9FF41C4EAFF42C4D9FF43C40E
:100A4A00DAFFDE50EE5C006E016A000E015A08D031
:100A5A000401404B412B424B432BD2D7006A016A17
:020A6A00120078
:0E0A6C00ADB202D00000FCD740C4AEFF1200B5
:040A7A00C58412001D
:100A7E0040C4E9FF41C4EAFFEE500401421905E10A
:100A8E0040C400F041C401F010D040C400F041C495
:100A9E0001F0404B412B00C0E9FF01C0EAFFEECF51
:0C0AAE0000F00052E5E1006A016A12004D
:0E0ABA00A8B202D00000FCD740C4A9FF120071
:100AC80026C4F6FF27C4F7FF28C4F8FF0900F5CFAE
:100AD80000F0005211E026C4F6FF27C4F7FF28C42F
:100AE800F8FF0900F5CF40F4BDDF010E0401262709
:0A0AF800000E27232823E4D7120084
:100B020004012A6B050E2A5D0AE22A512825E16EAC
:100B1200000E2921E26E200EE66E2A2BF3D72A510F
:100B22002825E16E000E2921E26EE66A2A072A5183
:100B320028252B6F000E29212C6F0A0E046E000E41
:100B4200056E26C400F027C401F07EDC08C000F068
:100B520009C001F0300E00262BC4E1FF2CC4E2FFD5
:100B620000C0E6FF0A0E046E000E056E26C400F0F9
:100B720027C401F069DC00C026F401C027F4000E8E
:100B8200011802E1000E001801E102D02A07CFD7B6
:020B920012004F
:100B940000C008F00150006E016A026A036A0B6A21
:100BA4000C6A016A026A036A960E036E0A6A00AE50
:100BB400E2EF05F0081E001E082AD8B4002A0A8EA7
:100BC40000C001F008C000F0086A026A68DC120084
:100BD4000D0E0401406F48DF0A0E0401406F44DF2C
:020BE4001200FD
:100BE60026C4F6FF27C4F7FF28C4F8FF0900F5CF8F
:100BF60000F0005211E026C4F6FF27C4F7FF28C410
:100C0600F8FF0900F5CF40F455DF010E0401262751
:0A0C1600000E27232823E4D7120064
:100C200079DCACC040F42CDC0401406B29DC000E04
:100C3000006E04012951005C02E12851100804E211
:100C4000100E286F000E296F0ED02851800F406FB4
:100C5000400716DC16D004012851C00F406F400732
:100C60000FDC0FD00ED0000E0401271902E1010E97
:100C70002619EBE0000E271902E1020E2619EBE01F
:100C8000F1D719EC02F0ACC040F440EC02F0400E99
:100C90000401406F40EC02F004012C6B2D6B2AC460
:100CA000E9FF2BC4EAFFEE5219E02AC4D9FF2BC496
:100CB000DAFFDE50800F406F40EC02F004012A4B57
:100CC0002B2B2C4B2D2B800E006E800E2D19005CD3
:100CD00002E12C51100801E201D0E1D7CEDE120072
:100CE00019DCACC040F440EC02F00401406B40EC75
:100CF00002F0020E0401406F40EC02F00DD0800EB5
:100D00000401406F40EC02F015D0C00E0401406FAA
:100D100040EC02F00FD00ED0000E0401271902E1C2
:100D2000010E2619ECE0000E271902E1020E261929
:100D3000ECE0F1D719EC02F0ACC040F440EC02F06A
:100D4000400E0401406F40EC02F00201516B526B07
:100D5000000E525D02E1270E515D09E2A00E040172
:100D6000406F40EC02F00201514B522BF1D719ECCD
:100D700002F0ACC040F440EC02F00401406B40ECE7
:100D800002F00DD0800E0401406F40EC02F015D04F
:100D9000C00E0401406F40EC02F00FD00ED0000EE8
:100DA0000401271902E1010E2619ECE0000E2719B3
:0E0DB00002E1020E2619ECE0F1D75FDE120020
:080DBE00067ED8EC02F01200E1
:100DC600000E0401271902E1000E261934E026C49C
:100DD600E9FF27C4EAFFEE522EE028C440F429C4F6
:100DE60041F4F3DD00C044F426C440F427C441F4C2
:100DF60028C442F429C443F405DE000E011802E1BA
:100E0600000E001805E126C400F027C401F015D035
:100E1600010E04012625406F000E2721416F28C4CC
:100E2600E9FF29C4EAFFEECF42F426DE00C026F42D
:0C0E360001C027F4C5D7006A016A120051
:100E42000050086E0150006E016A026A036A0B6A62
:100E52000C6A960E036E0A6A00C001F008C000F028
:0A0E6200086A026A51EC02F0120067
:100E6C00086A096A000E07620364BBEF07F00250C0
:100E7C0006180A6E075003267E0ED8A04CEF07F01A
:100E8C00035ED8B0C0EF07F050EF07F0035ED8A0B8
:100E9C00C5EF07F0028E068E02C00EF001C00BF0FB
:100EAC0000C00DF000500402F4CF0CF0015005020C
:100EBC00F4CF00F0F3CF08F00402F3500C26F450FA
:100ECC000822000E00220D500502F3500C26F4509F
:100EDC000822000E002202500402F3500826F4509F
:100EEC00002202500502016A000E0122F350002676
:100EFC00F45001220D500602F3500826F450002243
:100F0C00026A000E012202220B500602F350002648
:100F1C00F4500122000E02220E500602F35001265C
:100F2C00F450022202BEA3EF07F008360036013659
:100F3C0002360306D8B4C5EF07F0B6EF07F0D88039
:100F4C00800E08640030000E002201220222D8A07C
:100F5C00B6EF07F0023201320032034AC0EF07F05D
:100F6C000AAE029E000EC8EF07F0010EF5EC00F081
:100F7C00C8EF07F0020EE9EC00F0C8EF07F0040E22
:060F8C00FCEC00F0120075
:100F92000A6A0350D8A40A800750D8A40A820A50C9
:100FA200D8B42CEF08F0030AD8B4E5EF07F00AB082
:100FB200E0EF07F006AE2AEF08F028EF08F002AEE5
:100FC20028EF08F02AEF08F00250800B0A6E029E0A
:100FD2000650800B069E0A18D8B4F6EF07F00A50A6
:100FE200D8B428EF08F02AEF08F00750035CD8B411
:100FF20000EF08F0D8A01CEF08F022EF08F006502E
:10100200025CD8B40AEF08F0D8A01CEF08F022EF77
:1010120008F00550015CD8B414EF08F0D8A01CEF1A
:1010220008F022EF08F00450005CD8B42CEF08F06E
:10103200D8B022EF08F00A52D8B42AEF08F028EF0D
:1010420008F00A52D8B428EF08F02AEF08F0D88046
:0E1052001200D8901200D880D884120012002C
:10106000C26A070EC16EC18E26C400F00036009021
:10107000003600900050C212C2801EEC02F0C28204
:10108000C2A201D0FDD7C4CF01F0006AC350001244
:08109000000E0112C2901200D3
:101098000B6A0350D8B492EF08F002500A6E028E21
:1010A8008E0E035E03AE96EF08F0036C080E035C29
:1010B800D8A071EF08F0036E013602C001F0026A91
:1010C800080E035CD8A071EF08F0036E0136016AC0
:1010D8000350D8A4D8907BEF08F00350D8B47BEF26
:1010E80008F0D89002320132032E75EF08F00BBCDD
:1010F80001A088EF08F0D8A088EF08F0012AD8B43A
:10110800022A02BEA5EF08F00AAEABEF08F0021EF5
:10111800011E012AD8B4022AABEF08F0026A016A5C
:10112800ABEF08F00B800BAEAFEF08F0026A0AAE27
:10113800AFEF08F0FF0E026E016E0A360232AFEF13
:1011480008F0010E0C6E0BEC02F0B1EF08F0000E87
:101158000C6EB1EF08F0FF0E0C6E0150006E0250DD
:04116800016E120002
:10116C000450000A12E10550000A0FE10650000A73
:10117C000CE10750000A09E1FF0E006EFF0E016E34
:10118C007F0E026EFF0E036EA8D0086A096A075024
:10119C00D8B461EF09F00350D8B466EF09F00250EF
:1011AC0006180A6E028E068E0E6A02C008F001C086
:1011BC000CF000C00DF004500D5E0550D8A0053C9D
:1011CC000C5E0650D8A0063C085E086A0C6A0D6AD4
:1011DC00D8A0F8EF08F0D890023201320032083271
:1011EC00010E0E6E0750035ED8A005EF09F07E0EBF
:1011FC000E240326D8B06BEF09F00BEF09F07E0E2E
:10120C000E240326D8A070EF09F0180E0B6E0D36C5
:10121C000C3608360036013602360E360450005EA7
:10122C000550D8A0053C015E0650D8A0063C025ED5
:10123C0006340E120EA026EF09F00D8031EF09F0E6
:10124C00045000260550D8B0053C01260650D8B0F5
:10125C00062802260D900B2E0DEF09F057EF09F022
:10126C00D8900036013602360E360450005E05501A
:10127C00D8A0053C015E0650D8A0063C025E0634A0
:10128C000E10010B0D26D8B00C2AD8B4082AD8A4FD
:10129C0057EF09F008320C320D32032AD8B46BEF39
:1012AC0009F00AAE089E0850026E0C50016E0D50EB
:1012BC00006E73EF09F0010EABEC02F073EF09F066
:1012CC00020EF5EC00F073EF09F0040EE9EC00F0FF
:0C12DC0073EF09F0080EFCEC00F01200AB
:1012E8000401296B26C4E9FF27C4EAFFEECF28F4DE
:1012F8002851000A0FE028C440F436EC05F0040138
:10130800292B29512625E96E000E2721EA6EEECFFA
:0613180028F4EED71200DC
:10131E00086A080E0C6E003408360450085ED8B009
:0E132E0002D00826D89000360C2EF5D71200FB
:10133C00A39A2E6A2F6A010E2F5C02E1000E2E5C1E
:10134C000AE25B0E2E24E16E020E2F20E26EE66A9C
:10135C002E4A2F2AF0D7216A226A2E6A2F6AAACF28
:0E136C00C9F00001C96B6D6B6E6BA38A120095
:10137A002D0E0401406F040E416F2AC442F42BC49F
:10138A0043F42CC444F4AFEC02F08AEC02F0ACC093
:10139A0040F440EC02F00401406B40EC02F0000E15
:1013AA00006E04012951005C02E12851100804E290
:1013BA00100E286F000E296F10D02851800F406F31
:1013CA00400740EC02F017D004012851C00F406FCB
:1013DA00400740EC02F00FD00ED0000E040127198E
:1013EA0002E1010E2619E9E0000E271902E1020EB8
:1013FA002619EAE0F1D719EC02F0ACC040F440EC4F
:10140A0002F0400E0401406F40EC02F004013E6B12
:10141A003F6B2AC4F6FF2BC4F7FF2CC4F8FF090060
:10142A00F5CF00F0005221E02AC4F6FF2BC4F7FFE3
:10143A002CC4F8FF0900F5CF00F00050800F406F70
:10144A0040EC02F0010E04012A27000E2B232C2364
:10145A003E4B3F2B800E006E800E3F19005C02E16E
:10146A003E51100801E201D0D4D73DEC05F012003C
:10147A000FC404F010C405F004011351141124E040
:10148A00010E135F000E145B04C002F005C003F0E6
:10149A00044A052A11C400F012C401F0114B122BA0
:1014AA0000C0E9FF01C0EAFF02C0E1FF03C0E2FF9A
:1014BA00EECFE6FF02C0E9FF03C0EAFFEECF00F07D
:1014CA00005201E101D0D8D713C400F014C401F0CE
:1014DA00010E135F000E145B0050011008E004C0F7
:1014EA00E1FF05C0E2FFE66A044A052AEDD70FC408
:0814FA0000F010C401F0120023
:101502000401126B0FC4E9FF10C4EAFFEECF11F41D
:101512001151000A0FE011C440F45DEC05F0040122
:10152200122B12510F25E96E000E1021EA6EEECF3A
:0615320011F4EED71200D7
:10153800220E0C6E086A096A0A6A0B6A0C06D8B48D
:101548001FD0D8900B320A320932083203320232E5
:1015580001320032D8A0F2D70C06D8B409D0045012
:1015680008260550092206500A2207500B22EAD7FE
:10157800045008260550092206500A2207500B225B
:0215880012004F
:10158A000B6A0A6A096A086A0E6A03340836045042
:10159A00085E0550D8A0053C095E0650D8A0063C56
:1015AA000A5E0750D8A0073C0B5EE86AD8A0010E75
:1015BA000E5E0336070E0C6E0334083609360A36F9
:1015CA000B360E36045003A012D0085E0550D8A080
:1015DA00053C095E0650D8A0063C0A5E0750D8A012
:1015EA00073C0B5EE86AD8A0010E0E5E11D00826F1
:1015FA000550D8B0053C09260650D8B0063C0A2644
:10160A000750D8B0073C0B26E86AD8B0010E0E2660
:10161A0003360C2ED1D70234083609360A360B3671
:10162A000E36045003A012D0085E0550D8A0053C1F
:10163A00095E0650D8A0063C0A5E0750D8A0073CAF
:10164A000B5EE86AD8A0010E0E5E11D0082605507E
:10165A00D8B0053C09260650D8B0063C0A260750E1
:10166A00D8B0073C0B26E86AD8B0010E0E2602361F
:10167A00070E0C6E0234083609360A360B360E3659
:10168A00045002A012D0085E0550D8A0053C095E9D
:10169A000650D8A0063C0A5E0750D8A0073C0B5E4D
:1016AA00E86AD8A0010E0E5E11D008260550D8B0FF
:1016BA00053C09260650D8B0063C0A260750D8B081
:1016CA00073C0B26E86AD8B0010E0E2602360C2E0D
:1016DA00D1D70134083609360A360B360E3604508D
:1016EA0002A012D0085E0550D8A0053C095E06503B
:1016FA00D8A0063C0A5E0750D8A0073C0B5EE86AF1
:10170A00D8A0010E0E5E11D008260550D8B0053CAF
:10171A0009260650D8B0063C0A260750D8B0073C1E
:10172A000B26E86AD8B0010E0E260136070E0C6E9B
:10173A000134083609360A360B360E36045001A033
:10174A0012D0085E0550D8A0053C095E0650D8A004
:10175A00063C0A5E0750D8A0073C0B5EE86AD8A090
:10176A00010E0E5E11D008260550D8B0053C092698
:10177A000650D8B0063C0A260750D8B0073C0B26BC
:10178A00E86AD8B0010E0E2601360C2ED1D70034E5
:10179A00083609360A360B360E36045001A012D026
:1017AA00085E0550D8A0053C095E0650D8A0063C44
:1017BA000A5E0750D8A0073C0B5EE86AD8A0010E63
:1017CA000E5E11D008260550D8B0053C09260650F1
:1017DA00D8B0063C0A260750D8B0073C0B26E86A60
:1017EA00D8B0010E0E260036070E0C6E00340836ED
:1017FA0009360A360B360E36045000A012D0085E9F
:10180A000550D8A0053C095E0650D8A0063C0A5EE1
:10181A000750D8A0073C0B5EE86AD8A0010E0E5EFE
:10182A0011D008260550D8B0053C09260650D8B074
:10183A00063C0A260750D8B0073C0B26E86AD8B0FF
:10184A00010E0E2600360C2ED1D700B00ED0045051
:10185A0008260550D8B0053C09260650D8B0063CE3
:0C186A000A260750D8B0073C0B261200DD
:101876000401126B030E125D0AE212511025E16E8D
:10188600000E1121E26E200EE66E122BF3D71251D6
:101896001025E16E000E1121E26EE66A1207125162
:1018A6001025136F000E1121146F0A0E046E0FC45B
:1018B60000F032DD08C000F0300E002613C4E1FF50
:1018C60014C4E2FF00C0E6FF0A0E046E0FC400F067
:1018D60023DD00C00FF40050000A01E102D0120718
:0418E600DED7120037
:1018EA0028DD0FC426F410C427F411C428F4F3EC3D
:1018FA0005F0D60E0B6E110E0C6EE40E0D6E0D2E4B
:10190A00FED70C2EFCD70B2EFAD700005B0E040173
:10191A00266F020E276FE3DC125352E0090E406F66
:10192A0036EC05F05B0E0401266F020E276F230EBC
:10193A00286F000E296FE3EC06F0000E026E0150CC
:10194A00025C02E10050000803E201015E4B5F2BDA
:10195A005EC126F45FC127F4CFC128F4D0C129F4AF
:10196A0081EC05F0020E266F000E276F010E286F1C
:10197A00000E296FC40E2A6F560E2B6F000E2C6FA5
:10198A00F7DC020E266F000E276F070E286F000E77
:10199A00296FCFC12AF4D0C12BF410EC06F0600EE7
:1019AA00266F590E276F000E286F64EC05F0CFC121
:1019BA0026F4D0C127F493DC090E406F36EC05F00B
:0619CA00EAEC05F012003A
:1019D0009E96C5869EB601D0FDD7C9CF01F0040101
:1019E0000F51000A02E1C58A01D0C59A9E96C588AA
:0C19F0009EB601D0FDD701C000F012002F
:1019FC000FC404F010C405F004C002F005C003F0DD
:101A0C00044A052A11C400F012C401F00401114B60
:101A1C00122B00C0E9FF01C0EAFF02C0E1FF03C0C6
:101A2C00E2FFEECFE6FF02C0E9FF03C0EAFFEE5291
:0E1A3C0001E0E2D70FC400F010C401F0120068
:101A4A00020E0401266F000E276F70EC06F0010EDD
:0E1A5A000401266F000E276F70EC06F01200DC
:101A680004011551000805E3070E166F000E176FE5
:101A780012D01551160805E2170E186F000E196FCF
:101A880006D01551010F186F196B000E192318C4D1
:101A980016F419C417F416C420F417C421F41A6BE9
:101AA8001B6B046A056A066A076A0FC400F010C453
:101AB80001F011C402F012C403F0C9EC07F0010EE2
:101AC800D8B0000E006E005209E013C4E1FF14C440
:101AD800E2FF2D0EE66E134B142B117F0FC404F09A
:101AE80010C405F011C406F012C407F0006A016AB8
:101AF800026A036AC9EC07F0010ED8B0000E006E46
:101B0800005237E0000E046E000E056E000E066EE1
:101B18007F0E076E0FC400F010C401F011C402F06C
:101B280012C403F0C9EC07F0010ED8B0000E006E25
:101B380000521FE00FC400F010C401F011C402F0FD
:101B480012C403F0000E046E000E056E200E066E21
:101B5800820E076E36EC07F000C00FF401C010F4D7
:101B680002C011F403C012F4010E1A5F000E1B5BD1
:101B7800C9D7000E046E000E056E200E066E820E8A
:101B8800076E0FC400F010C401F011C402F012C4B3
:101B980003F0C9EC07F0000ED8B0010E006E005239
:101BA8001EE0000E046E000E056E200E066E820EFC
:101BB800076E0FC400F010C401F011C402F012C483
:101BC80003F0B6EC08F000C00FF401C010F402C036
:101BD80011F403C012F404011A4B1B2BCAD71A5173
:101BE80020271B512123010E1C6F000E1D6F000EB4
:101BF800226F000E236F000E246F7F0E256F800E5C
:101C08001D19006E800E2119005C02E120511C5D37
:101C18001EE2000E046E000E056E200E066E820E89
:101C2800076E22C400F023C401F024C402F025C4C6
:101C380003F0B6EC08F000C022F401C023F402C09F
:101C480024F403C025F404011C4B1D2BD8D7000E27
:101C5800046E000E056E000E066E800E076E22C41E
:101C680000F023C401F024C402F025C403F0B6EC4C
:101C780008F00FC404F010C405F011C406F012C433
:101C880007F0D8EC02F000C00FF401C010F402C055
:101C980011F403C012F4000E046E000E056E200E3F
:101CA800066E820E076EC9EC07F0000ED8B0010E62
:101CB800006E00520BE0000E04010F6F000E106F53
:101CC800000E116F7F0E126F1A4B1B2B0401800E32
:101CD8001B19006E800E005C02E1000E1A5D38E2EE
:101CE80013C4E1FF14C4E2FF300EE66E134B142B4D
:101CF80013C4E1FF14C4E2FF2E0EE66E134B142B3F
:101D0800800E2119006E800E005C02E1000E205D3D
:101D180004E220511A5F21511B5BFF0E1C6FFF0E5E
:101D28001D6F800E1B19006E800E1D19005C02E1EC
:101D38001C511A5D0DE213C4E1FF14C4E2FF300E1A
:101D4800E66E134B142B010E1C5F000E1D5BE9D7CA
:101D58001C6B1D6B800E1D19006E800E2119005C16
:101D680002E120511C5D63E20FC400F010C401F0D1
:101D780011C402F012C403F04CEC08F000C01EF4C9
:101D880001C01FF4300E002613C4E1FF14C4E2FFA3
:101D980000C0E6FF134B142B1D511B1902E11A5109
:101DA8001C1908E113C4E1FF14C4E2FF2E0EE66E0D
:101DB800134B142B1EC400F01FC401F0CAEC05F02D
:101DC80000C022F401C023F402C024F403C025F4A7
:101DD80000C004F001C005F002C006F003C007F01F
:101DE8000FC400F010C401F011C402F012C403F0D3
:101DF800DFEC06F000C00FF401C010F402C011F4CB
:101E080003C012F4000E046E000E056E200E066E5E
:101E1800820E076E36EC07F000C00FF401C010F414
:101E280002C011F403C012F41C4B1D2B93D713C42A
:0A1E3800E1FF14C4E2FFE66A1200A5
:101E42000FC404F010C405F004C0E9FF05C0EAFFA6
:101E5200EE5203E0044A052AF7D704C002F005C097
:101E620003F0044A052A11C400F012C401F004016F
:101E7200114B122B00C0E9FF01C0EAFF02C0E1FFD3
:101E820003C0E2FFEECFE6FF02C0E9FF03C0EAFFB4
:101E9200EE5201E0E2D70FC400F010C401F01200CC
:101EA200800E0401106F116B126B300E136F300E27
:101EB200146F300E156F300E166F300E176F300E16
:101EC200186F300E196F300E1A6F1B6B800E1219BD
:101ED200006E800E005C02E1080E115D13E21051EB
:101EE2000F15016E0150000808E2130E1125E16E74
:101EF200040E1221E26E310EE66E1033109F114B6A
:101F0200122BE4D71B6B130E006E040E016E12002F
:101F1200020E0401266F30EC08F0060E005C056E1E
:101F2200000E0158066E05C0AEF106C0AFF1070EF5
:101F320001015A15036E5BC104F0000E041603C0C2
:101F420000F004C001F00036009001364A0E002471
:101F5200E16E010E0120E26E05C0E6FF06C0E6FF5B
:101F62005A4B5B2B5C6B5D6B0201516B526B000E2B
:101F7200525D02E1080E515D16E251C200F052C2FA
:101F820001F00036009001364A0E0024D96E010E8F
:101F92000120DA6EDE5001015C27DE505D23020172
:101FA200514B522BE4D75CC100F05DC101F021EC32
:101FB20007F0000E046E000E056E250E066E7A0EF8
:081FC200076E36EC07F0120077
:101FCA008AEC02F0ACC040F440EC02F00401406B31
:101FDA0040EC02F0800E006E800E04011219005CC3
:101FEA0002E11151100804E2100E116F000E126F77
:101FFA0010D01151800F406F400740EC02F017D00B
:10200A0004011151C00F406F400740EC02F00FD09D
:10201A000ED0000E0401101902E1010E0F19E9E0B9
:10202A00000E101902E1020E0F19EAE0F1D719ECBD
:10203A0002F0ACC040F440EC02F0400E0401406FE4
:10204A0040EC02F013C440F440EC02F03DEC05F021
:02205A00120072
:10205C00A10E0401266F570E276F000E286F64EC3B
:10206C0005F0D1C30FF48D0E0401106F030E116F28
:10207C003BEC0CF08D0E266F030E276F74EC09F001
:10208C008AEC02F0D1C340F440EC02F00050000A9C
:10209C000CE0ED0E0401266F570E276F000E286F13
:1020AC0064EC05F00301D26B0CD09C0E0401266F7E
:1020BC00580E276F000E286F64EC05F0010E03011B
:1020CC00D26F3DEC05F0EAEC05F0D2C300F0120043
:1020DC00949894968B988B9694889486C79EC79C5C
:0620EC00380EC66E120062
:1020F200FF0E0101BB6FFF0EBC6FFF0EBD6FFF0E27
:0E210200BE6FC26A070EC16EC18EC28012008F
:10211000FF0E986EEF0E926EBF0E946EC088F90E91
:10212000C16EFF0EC26EC098938093849280959486
:10213000988693869596F19E9A8A92988988958E2C
:0E214000998695989698959C8C988D9812008B
:10214E000900F5CFE6FF0006FBE10106F9E11200FA
:10215E000301D76BD86B000ED85D02E10A0ED75D76
:10216E000BE2D751D525E16ED851D621E26E200E65
:10217E00E66ED74BD82BEFD7D751D525E16ED85178
:10218E00D621E26EE66A010ED75F000ED85BD751FC
:10219E00D525D96FD851D621DA6F0A0E046E000EEE
:1021AE00056E066E076ED1C300F0D2C301F0D3C325
:1021BE0002F0D4C303F0C5EC0AF008C000F009C069
:1021CE0001F00AC002F00BC003F0300E0026D9C396
:1021DE00E1FFDAC3E2FF00C0E6FF0A0E046E000E56
:1021EE00056E066E076ED1C300F0D2C301F0D3C3E5
:1021FE0002F0D4C303F0C5EC0AF000C0D1F301C065
:10220E00D2F302C0D3F303C0D4F3000E046E03184E
:10221E0008E10450021805E10450011802E10050D3
:10222E00000A01E105D0010ED75F000ED85BAFD7D3
:02223E0012008C
:10224000BA0E0201536F0A0E546F400E556F040E02
:10225000566FFF0E0101C36FFF0EC46F000EC56FF6
:10226000000EC66FFF0EBF6FFF0EC06F000EC16F76
:10227000000EC26FFF0EC76FFF0EC86F000EC96F52
:10228000000ECA6FA88A900E9C6E98849892A4AA99
:0A22900003D0AACF00F0FBD7120024
:10229A006C0E0201536F0A0E546F400E556F040EF6
:1022AA00566FFF0E0101C36FFF0EC46F000EC56F9C
:1022BA00000EC66FFF0EBF6FFF0EC06F000EC16F1C
:1022CA00000EC26FFF0EC76FFF0EC86F000EC96FF8
:1022DA00000ECA6FAD8A900EAC6E948E949C9EAA24
:0A22EA0003D0AFCF00F0FBD71200C5
:1022F400010E0401266F000E276F70EC06F0D10E5C
:102304000101CF6F010ED06FCFC140F4D0C141F4B1
:10231400440E0401426F590E436F000E446FAFEC3C
:1023240002F0B7C10FF4B8C110F4B9C111F4BAC1C5
:1023340012F48D0E0401136F030E146F020E156F49
:1023440034EC0DF0CFC10FF4D0C110F48D0E116F29
:10235400030E126F74DDCFC140F4D0C141F4E8EC38
:1023640004F000C051F201C052F257C20FF48D0EB6
:10237400106F030E116F3BEC0CF0CFC10FF4D0C102
:1023840010F48D0E116F030E126F59DD100E010142
:10239400CF25E16E000ED021E26EE66A010E040143
:1023A400266F000E276F010E286F000E296FCFC114
:1023B4002AF4D0C12BF410EC06F08D0E406F030EFE
:1023C400416F900E426F570E436F000E446FAFEC97
:1023D40002F0000E80B0010E0301906F300E9027C2
:1023E400000E0101B4B5010E0301966F300E96275D
:1023F400000E0101B4BB010E03019B6F300E9B273D
:102404009D6B020E0401266F000E276F70EC06F020
:10241400020E0401266F000E276F010E286F000EB6
:10242400296F8D0E2A6F030E2B6F10EC06F012002D
:10243400D596D584D582D580D59AD59C480ED76EAD
:10244400E50ED66EF2940301CD6BCE6BCF6BD06BE1
:08245400F184F28AD58E12001A
:10245C008AEC02F0400E0401406F40EC02F0120EC8
:10246C000401406F40EC02F0D1C340F440EC02F0A8
:06247C003DEC05F012002A
:10248200070E0401266F530E276F000E286F64ECAF
:1024920005F0D1C326F4D2C327F474EC09F0EAECB8
:1024A20005F09EEC09F04A0E0401266F540E276FC8
:1024B200000E286F64EC05F0010E0401266F000E79
:1024C200276F010E286F000E296F7F0E2A6F570E9D
:1024D2002B6F000E2C6FBDEC09F00F0E006E000E7C
:1024E200016E026E036E59C204F05AC205F0000E6C
:1024F20002015ABFFF0E066E076E9CEC0AF0E30E55
:1025020000240401266F500E0120276F000E0220C6
:10251200286F64EC05F0EAEC05F05D0E0401406FF3
:10252200030E416FE70E426F580E436F000E446F69
:10253200AFEC02F0650E0401406F030E416F0F0E07
:10254200006E000E016E026E036E59C204F05AC292
:1025520005F0000E02015ABFFF0E066E076E9CECDC
:102562000AF0E30E00240401426F500E0120436F73
:10257200000E0220446FAFEC02F0020E0401266F3F
:10258200000E276F70EC06F0020E0401266F000E9B
:10259200276F010E286F000E296F0F0E006E000EBE
:1025A200016E026E036E59C204F05AC205F0000EAB
:1025B20002015ABFFF0E066E076E9CEC0AF0E30E94
:1025C200002404012A6F500E01202B6F000E0220FE
:1025D2002C6FBDEC09F05D0E0F6F030E106F81ECD6
:1025E2000AF00D0E406F5DEC05F09EEC09F0B70E9F
:1025F2000B6EA10E0C6EC30E0D6E0D2EFED70C2EA1
:10260200FCD70B2EFAD7000000005B0E0401266FE8
:10261200020E276F74EC09F03E0E02015B6F9EEC16
:1026220009F0DD0E0401266F530E276F000E286F8E
:1026320064EC05F0CFC10FF4D0C110F481EC0AF0C4
:102642000D0E406F5DEC05F00A0E0401406F5DEC6B
:1026520005F01A0E0401406F5DEC05F09EEC09F0E6
:10266200020E0A6E120E0B6EF20E0C6E240E0D6E20
:102672000D2EFED70C2EFCD70B2EFAD70A2EF8D72A
:1026820000005B0E0401266F020E276F74EC09F046
:102692005B0E266F020E276FAD0E286F000E296F9C
:1026A200E3EC06F000C05BF301C05CF3000E026EC7
:1026B2000150025C02E1005000080AE27E0E0401B1
:1026C200266F540E276F000E286F64EC05F064D05D
:1026D2005B0E0401266F020E276FB30E286F000EE9
:1026E200296FE3EC06F000C05BF301C05CF3000E5F
:1026F200026E0150025C02E1005000084DE2B10E90
:102702000401266F570E276F000E286F64EC05F048
:102712005B0E0401266F020E276FBC0E286F000E9F
:10272200296FE3EC06F000C05BF301C05CF3CFC19C
:102732000FF4D0C110F400C011F401C012F40A0E5B
:102742000401136F000E146F3DEC0AF0CFC126F4A2
:10275200D0C127F474EC09F0EAEC05F01A0E03017B
:102762005B25E16E000E5C21E26EE66A020E040158
:10277200266F000E276F70EC06F0020E0401266F22
:10278200000E276F010E286F000E296FCFC12AF4A9
:10279200D0C12BF410EC06F0EAEC05F09EEC09F047
:0227A200120023
:1027A400D10E0101CF6F010ED06FD1C3E1FFD2C3AF
:1027B400E2FFE66A0301D36BD1C340F4D2C341F410
:1027C4000A0E0401426F550E436F000E446FAFECC6
:1027D40002F0D1C340F4D2C341F4E8EC04F000C0E9
:1027E4009DF001C09EF00101B4A99DD00301D36BFB
:1027F400D30E0401406F030E416F170E426F580E43
:10280400436F000E446FAFEC02F0B3C10FF451EC10
:102814000FF000C011F401C012F4D70E0F6F030EB5
:10282400106FFEEC0CF0D30E406F030E416FE8EC1A
:1028340004F000C09DF001C09EF0D30E0024E16EB0
:10284400030E0120E26E0D0EE66E00019D4B9E2BE1
:10285400D30E9D25E16E030E9E21E26E0A0EE66EF6
:102864009D4B9E2BD30E9D25E16E030E9E21E26EA1
:10287400E66AD1C30FF4D2C310F4D30E0401116F6E
:10288400030E126F21EC0FF00301D36BD30E04017E
:10289400406F030E416F310E426F580E436F000EAE
:1028A400446FAFEC02F0B0C10FF451EC0FF000C074
:1028B40011F401C012F4D70E0F6F030E106FFEEC6B
:1028C4000CF0D30E406F030E416FE8EC04F000C02F
:1028D4009DF001C09EF0D30E0024E16E030E012092
:1028E400E26E0D0EE66E00019D4B9E2BD30E9D25D0
:1028F400E16E030E9E21E26E0A0EE66E9D4B9E2B48
:10290400D30E9D25E16E030E9E21E26EE66AD1C3CD
:102914000FF4D2C310F4D30E0401116F030E126F1F
:1029240021EC0FF00FD00301D36BD30E0401406FE1
:10293400030E416F170E426F560E436F000E446F25
:10294400AFEC02F00301D36BD30E0401406F030E0E
:10295400416F180E426F590E436F000E446FAFEC77
:1029640002F0D30E0401406F030E416FE8EC04F053
:1029740000C09DF001C09EF0D30E0024E16E030E52
:102984000120E26E006A83BE002A300E002600C0D9
:10299400E6FF00019D4B9E2BD30E9D25E16E030E99
:1029A4009E21E26E0D0EE66E9D4B9E2BD30E9D2551
:1029B400E16E030E9E21E26E0A0EE66E9D4B9E2B87
:1029C400D30E9D25E16E030E9E21E26EE66AD1C30D
:1029D4000FF4D2C310F4D30E0401116F030E126F5F
:1029E40021EC0FF00301D36BD30E0401406F030EEF
:1029F400416F200E426F590E436F000E446FAFECCF
:102A040002F0D30E0401406F030E416FE8EC04F0B2
:102A140000C09DF001C09EF0D30E0024E16E030EB1
:102A24000120E26E006A87B6002A300E002600C03C
:102A3400E6FF00019D4B9E2BD30E9D25E16E030EF8
:102A44009E21E26E0D0EE66E9D4B9E2BD30E9D25B0
:102A5400E16E030E9E21E26E0A0EE66E9D4B9E2BE6
:102A6400D30E9D25E16E030E9E21E26EE66AD1C36C
:102A74000FF4D2C310F4D30E0401116F030E126FBE
:102A840021EC0FF00301D36BD30E0401406F030E4E
:102A9400416F000E426F590E436F000E446FAFEC4E
:102AA40002F0D30E0401406F030E416FE8EC04F012
:102AB40000C09DF001C09EF0D30E0024E16E030E11
:102AC4000120E26E006A83B8002A300E002600C09E
:102AD400E6FF00019D4B9E2BD30E9D25E16E030E58
:102AE4009E21E26E0D0EE66E9D4B9E2BD30E9D2510
:102AF400E16E030E9E21E26E0A0EE66E9D4B9E2B46
:102B0400D30E9D25E16E030E9E21E26EE66AD1C3CB
:102B14000FF4D2C310F4D30E0401116F030E126F1D
:102B240021EC0FF00301D36BD30E0401406F030EAD
:102B3400416FF00E426F580E436F000E446FAFECBE
:102B440002F0D30E0401406F030E416FE8EC04F071
:102B540000C09DF001C09EF0D30E0024E16E030E70
:102B64000120E26E006A84B8002A300E002600C0FC
:102B7400E6FF00019D4B9E2BD30E9D25E16E030EB7
:102B84009E21E26E0D0EE66E9D4B9E2BD30E9D256F
:102B9400E16E030E9E21E26E0A0EE66E9D4B9E2BA5
:102BA400D30E9D25E16E030E9E21E26EE66AD1C32B
:102BB4000FF4D2C310F4D30E0401116F030E126F7D
:102BC40021EC0FF00301D36B010E0401266F30ECEE
:102BD40008F000C0B1F101C0B2F10150020802E1F5
:102BE400005000080EE2D30E0401406F030E416F43
:102BF4005E0E426F560E436F000E446FAFEC02F050
:102C04000DD0D30E0401406F030E416F6D0E426F61
:102C1400590E436F000E446FAFEC02F0D30E040163
:102C2400406F030E416FE8EC04F000C09DF001C05A
:102C34009EF0B1C126F4B2C127F4D30E0024286F4C
:102C4400030E0120296F81EC05F0D30E406F030EB3
:102C5400416FE8EC04F000C09DF001C09EF0D30E7B
:102C64000024E16E030E0120E26E0D0EE66E0001FB
:102C74009D4B9E2BD30E9D25E16E030E9E21E26E8D
:102C84000A0EE66E9D4B9E2BD30E9D25E16E030E20
:102C94009E21E26EE66AD1C30FF4D2C310F4D30EC0
:102CA4000401116F030E126F21EC0FF00301D36BBB
:102CB40089EC0FF000C0B7F101C0B8F102C0B9F15E
:102CC40003C0BAF1D30E0401406F030E416F100E1E
:102CD400426F590E436F000E446FAFEC02F0D30EF7
:102CE4000401406F030E416FE8EC04F000C09DF056
:102CF40001C09EF0B7C10FF4B8C110F4B9C111F40A
:102D0400BAC112F4D30E0024136F030E0120146F02
:102D1400020E156F34EC0DF0D30E406F030E416FAD
:102D2400E8EC04F000C09DF001C09EF0D30E002436
:102D3400E16E030E0120E26EB00EE66E00019D4BC3
:102D44009E2BD30E9D25E16E030E9E21E26E430E53
:102D5400E66E9D4B9E2BD30E9D25E16E030E9E21A8
:102D6400E26EE66AD1C30FF4D2C310F4D30E0401A9
:102D7400116F030E126F21EC0FF00301D36BD30E0E
:102D84000401406F030E416F920E426F580E436F61
:102D9400000E446FAFEC02F0D1C30FF4D2C310F4B1
:102DA400D30E0401116F030E126F21EC0FF0030117
:102DB400D36BD1C340F4D2C341F4E8EC04F000C0B7
:082DC4009DF001C09EF0120019
:102DCC009D989D9A00019D6B9E6B000E9E5D02E18D
:102DDC00800E9D5D0AE2CA0E9D25E16E000E9E21BD
:102DEC00E26EE66A9D4B9E2BF0D79D6B9E6B616BE2
:102DFC00626BAFCF60F0606B746B756B9D8A120069
:102E0C008AEC02F0ACC040F440EC02F0400E04013D
:102E1C00406F40EC02F00A0E0401406F40EC02F0EF
:102E2C000401406B40EC02F03DEC05F08AEC02F042
:102E3C00400E0401406F40EC02F00401406B40EC8A
:102E4C0002F00401406B40EC02F0FF0E0401406FF5
:102E5C0040EC02F00401406B40EC02F0FF0E040168
:102E6C00406F40EC02F03DEC05F08AEC02F0400EB5
:102E7C000401406F40EC02F00D0E0401406F40EC79
:102E8C0002F0FF0E0401406F40EC02F03DEC05F047
:022E9C00120022
:102E9E000301D36BD46B1F0E0B6E710E0C6E1E0ED8
:102EAE000D6E0D2EFED70C2EFCD70B2EFAD7000072
:102EBE008AEC02F0ACC040F440EC02F000C0D1F35A
:102ECE00000E0301D26F000ED21902E1000ED119CD
:102EDE0005E0D3C300F0D4C301F0E6D0D34BD42B1E
:102EEE000D0E0B6E2D0E0C6ED70E0D6E0D2EFED71B
:102EFE000C2EFCD70B2EFAD7000000000401406BFD
:102F0E0040EC02F000C0D1F3000E0301D26F800E30
:102F1E00006E800ED219005C02E1D151000805E26C
:102F2E00D3C300F0D4C301F0BFD0D34BD42B240EA7
:102F3E000401406F40EC02F00C0E0401406F40ECB7
:102F4E0002F0060E0401406F40EC02F0250E040163
:102F5E00406F40EC02F0060E0401406F40EC02F0B0
:102F6E00110E0401406F40EC02F0420E0401406F5E
:102F7E0040EC02F0960E0401406F40EC02F0240E7D
:102F8E000401406F40EC02F000C0D1F3000E0301CB
:102F9E00D26F800E006E800ED219005C02E1D1510C
:102FAE00000805E2D3C300F0D4C301F07DD0D34BAB
:102FBE00D42B0C0E0401406F40EC02F000C0D1F394
:102FCE00000E0301D26F800E006E800ED219005CCF
:102FDE0002E1D151000805E2D3C300F0D4C301F0E1
:102FEE0063D0D34BD42B060E0401406F40EC02F09D
:102FFE0000C0D1F3000E0301D26F800E006E800E62
:10300E00D219005C02E1D151000805E2D3C300F0F1
:10301E00D4C301F049D0D34BD42B020E0401406F20
:10302E0040EC02F000C0D1F3000E0301D26F800E0F
:10303E00006E800ED219005C02E1D151000805E24B
:10304E00D3C300F0D4C301F02FD0D34BD42B010E39
:10305E000401406F40EC02F000C0D1F3000E0301FA
:10306E00D26F800E006E800ED219005C02E1D1513B
:10307E00000805E2D3C300F0D4C301F015D0070E4B
:10308E000B6E170E0C6E6A0E0D6E0D2EFED70C2EDD
:10309E00FCD70B2EFAD700003DEC05F0D34BD42B0A
:0A30AE00D3C300F0D4C301F01200F8
:1030B8000301D16BD26B0001766B776B780E04013C
:1030C800266F550E276F000E286F64EC05F09EECF6
:1030D80009F08A0E0401266F590E276F000E286F1B
:1030E800F3EC05F03D0E0B6EE10E0C6E3F0E0D6E0F
:1030F8000D2EFED70C2EFCD70B2EFAD700000000A1
:10310800000E00016E1902E1010E6D1934E15B0E2B
:103118000401266F020E276F6A0E286F000E296FB2
:10312800E3EC06F0000E026E0150025C02E1005072
:10313800000821E2150E0301D16F000ED26F010EB7
:103148000001766F000E776F5B0E0401266F020E8A
:10315800276F74EC09F0020E266F000E276F010E20
:10316800286F000E296FF70E2A6F560E2B6F000E70
:103178002C6FBDEC09F01F0E0B6E710E0C6E1E0E3F
:103188000D6E0D2EFED70C2EFCD70B2EFAD7000095
:103198000301D14BD22B800ED219006E800E005C39
:1031A80002E1140ED15D08E2000E0001771902E178
:0A31B800000E761901E18BD712001A
:1031C2008AEC02F0400E0401406F40EC02F04F0E18
:1031D2000D6E0D2EFED700000000130E0401406F8D
:1031E20040EC02F03DEC05F08AEC02F0410E0401E5
:1031F200406F40EC02F004010F6BE8EC0CF000C0F1
:0C320200D1F33DEC05F0D1C300F0120048
:10320E00010E0401266F000E276F010E286F000EAF
:10321E00296FE60E2A6F560E2B6F000E2C6FBDEC2B
:10322E0009F08D8801015E6B5F6BB487830E04011C
:10323E00266F530E276F000E286F64EC05F0FB0E01
:10324E0004010F6F570E106F000E116F000E01016B
:10325E00B4B7010E0401126F75EC0CF0550E04019B
:10326E00266F500E276F000E286F64EC05F0A60E29
:10327E0004010F6F580E106F000E116F000E01013A
:10328E00B4B7010E0401126F75EC0CF08C0E040134
:10329E00266F510E276F000E286F64EC05F0B00EEE
:1032AE0004010F6F580E106F000E116F000E01010A
:1032BE00B4B7010E0401126F75EC0CF0650E04012B
:1032CE00266F510E276F000E286F64EC05F04B0E23
:1032DE0004010F6F580E106F000E116F000E0101DA
:1032EE00B4B7010E0401126F75EC0CF0B80E0401A8
:1032FE00266F4F0E276F000E286F64EC05F0360E0A
:10330E0004010F6F550E106F000E116F000E0101AC
:10331E00B4B7010E0401126F75EC0CF05C0E0B6E5F
:10332E00510E0C6E600E0D6E0D2EFED70C2EFCD7B0
:10333E000B2EFAD70000290E0401266F560E276FAA
:10334E00000E286F64EC05F025EC0DF0010E040163
:10335E00266F000E276F010E286F000E296FA20E2A
:10336E002A6F560E2B6F000E2C6FBDEC09F05EC14E
:10337E0026F45FC127F4CFC128F4D0C129F481EC23
:10338E0005F0CFC126F4D0C127F474EC09F0020E7B
:10339E00266F000E276F70EC06F0590E0401266F93
:1033AE00590E276F000E286F64EC05F0020E040113
:1033BE00266F000E276F010E286F000E296FD50E97
:1033CE002A6F560E2B6F000E2C6FBDEC09F0020EFD
:1033DE000F6F000E106F030E116F000E126F300E76
:1033EE0001015E250401136FE5EC0FF05EC100F0E4
:0633FE005FC101F01200A6
:10340400C7EC2CF088EC10F08D88D10E0101CF6F41
:10341400010ED06FD16B03018D6B02015B6B010157
:10342400B16BB26B606B616B626B636B5E6B5F6B9A
:10343400B487B495B49BB48FB49D8C9C0201596B32
:103444005A6B8D988C88800E0101646FBB0E656F7A
:10345400000E666F676F800E0301D16FBB0ED26FD3
:10346400000ED36F000ED46FCFC1D5F3D0C1D6F305
:10347400AFEC10F07E86020E7F6E700EB06EAD84DF
:103484004DEC11F00C0E0401406F36EC05F01F0EEC
:103494000B6E710E0C6E1E0E0D6E0D2EFED70C2EC5
:1034A400FCD70B2EFAD70000EAEC05F08C987C864A
:1034B400020E7D6E700EAB6EA88420EC11F07B0EB4
:1034C4000401266F4F0E276F000E286F64EC05F081
:1034D400AC0E0401266F4E0E276F000E286F64ECAD
:1034E40005F0620E0401266F4E0E276F000E286F42
:1034F40064EC05F03B0E0401266F510E276F000E9D
:10350400286F64EC05F0D50E0401266F580E276F62
:10351400000E286F64EC05F0CFC126F4D0C127F467
:1035240074EC09F0EAEC05F0230E0401406F36EC6C
:1035340005F0EAEC05F0020E0A6E310E0B6E620E17
:103544000C6E450E0D6E0D2EFED70C2EFCD70B2ED9
:10355400FAD70A2EF8D7240E0401406F36EC05F092
:10356400EAEC05F079EC10F03E0E0401266F580EDB
:10357400276F000E286F64EC05F0A20E0401266F7D
:10358400550E276F000E286F64EC05F0780EC86E98
:103594006EEC10F0070E0B6E170E0C6E6A0E0D6EAD
:1035A4000D2EFED70C2EFCD70B2EFAD70000FD0EE5
:1035B4000401266F510E276F000E286F64EC05F08E
:1035C400010E0401266F30EC08F000C0B1F101C017
:1035D400B2F100C026F401C027F4CFC128F4D0C151
:1035E40029F481EC05F0CFC126F4D0C127F474ECA2
:1035F40009F0090E406F36EC05F001015C6B5D6B60
:10360400020E0401266F30EC08F000C0AEF101C0D8
:10361400AFF100C026F401C027F4CFC128F4D0C113
:1036240029F481EC05F0CFC126F4D0C127F474EC61
:1036340009F0EAEC05F00201516B526B000E525D89
:1036440002E1080E515D14E251C200F052C201F0D1
:103654000036009001364A0E0024E16E010E01206E
:10366400E26EAEC1E6FFAFC1E6FF514B522BE6D787
:1036740001015A6B5B6B3C0E0401266F4F0E276FE2
:10368400000E286F64EC05F0740E0001AC6F300E70
:103694000401266F540E276F000E286F64EC05F0AA
:1036A400ACC0D1F32EEC10F001016A6B6B6B4FECE4
:1036B40017F000C06AF101C06BF1070E0B6E170E14
:1036C4000C6E6A0E0D6E0D2EFED70C2EFCD70B2E33
:1036D400FAD7000025EC0DF0CA0E0401266F550E32
:1036E400276F000E286F64EC05F06AC126F46BC1E5
:1036F40027F4CFC128F4D0C129F481EC05F0AF0E32
:10370400266F540E276F000E286F64EC05F0CFC1AE
:1037140026F4D0C127F474EC09F0EAEC05F0010EAC
:103724000401266F000E276F70EC06F0010E0401F1
:10373400266F000E276F010E286F000E296F3B0EB7
:103744002A6F570E2B6F000E2C6FBDEC09F0640E20
:10375400266F530E276F000E286F64EC05F0400EA1
:103764000301D16F2EEC10F000C060F006EC17F0EE
:103774000101B06B00016051010A14E1020E040161
:10378400266F000E276F010E286F000E296F2A0E78
:103794002A6F570E2B6F000E2C6FBDEC09F0010140
:1037A400B48913D00101B499020E0401266F000EEE
:1037B400276F010E286F000E296F4C0E2A6F570ECB
:1037C4002B6F000E2C6FBDEC09F00001606B3D0EF9
:1037D4000B6EE10E0C6E3F0E0D6E0D2EFED70C2EF1
:1037E400FCD70B2EFAD700000000C80E0401266F88
:1037F400520E276F000E286F64EC05F03D0E0B6E21
:10380400E10E0C6E3F0E0D6E0D2EFED70C2EFCD766
:103814000B2EFAD7000000008C84020E0A6E310EC3
:103824000B6E620E0C6E450E0D6E0D2EFED70C2E19
:10383400FCD70B2EFAD70A2EF8D78C943D0E0B6EBC
:10384400E10E0C6E3F0E0D6E0D2EFED70C2EFCD726
:103854000B2EFAD7000000008C96C60E0401266FCA
:10386400540E276F000E286F64EC05F09EEC09F0EF
:10387400AC8EAC86AC969C96D08EA38AF28CF28EDB
:1038840019DC000E0001771902E1010E76190AE134
:10389400050E0401266F560E276F000E286F64EC88
:1038A40005F019D0260E0401266F530E276F000E63
:1038B400286F64EC05F08C783D0E0B6EE10E0C6EF7
:1038C4003F0E0D6E0D2EFED70C2EFCD70B2EFAD705
:1038D40000000000F0D7D10E0101CF6F010ED06FB0
:1038E40094DC00C05EF101C05FF1000E011802E13A
:1038F400050E00180CE1730E0401266F590E276F94
:10390400000E286F64EC05F00101B48558D0520E06
:103914000401266F590E276F000E286F64EC05F022
:103924000101B495100E0401266F510E276F000E8D
:10393400286F64EC05F025EC0DF0010E0401266FF0
:10394400000E276F010E286F000E296F6E0E2A6F6E
:10395400570E2B6F000E2C6FBDEC09F0010E0F6F8C
:10396400000E106F0F0E116F000E126F300E01015A
:103974005E250401136FE5EC0FF0020E0401266FBF
:10398400000E276F010E286F000E296F5D0E2A6F3F
:10399400570E2B6F000E2C6FBDEC09F0020E0A6E51
:1039A400310E0B6E620E0C6E450E0D6E0D2EFED793
:1039B4000C2EFCD70B2EFAD70A2EF8D7B3D7EAEC85
:1039C40005F07A0E0B6EC10E0C6E810E0D6E0D2E6F
:1039D400FED70C2EFCD70B2EFAD70000000079EC92
:1039E40010F08C98210E0401266F520E276F000EE2
:1039F400286F64EC05F0010E0401266F30EC08F02A
:103A040000C0B1F101C0B2F100C026F401C027F436
:103A1400CFC128F4D0C129F481EC05F0CFC126F43C
:103A2400D0C127F474EC09F0090E406F36EC05F0B0
:103A3400020E0401266F30EC08F000C0AEF101C0A4
:103A4400AFF100C026F401C027F4CFC128F4D0C1DF
:103A540029F481EC05F0CFC126F4D0C127F474EC2D
:103A640009F0EAEC05F0D10E0101CF6F010ED06F21
:103A7400450E0401266F520E276F000E286F64EC6A
:103A840005F0CFC1D1F3D0C1D2F3D2EC13F000C012
:103A940068F101C069F1EAEC05F0070E0B6E170E30
:103AA4000C6E6A0E0D6E0D2EFED70C2EFCD70B2E4F
:103AB400FAD700008D9801015E6B5F6BB497B49BDD
:103AC4008C9CDD0E0401266F540E276F000E286FA8
:103AD40064EC05F0E6EC16F00201576B586BD10E5E
:103AE4000101CF6F010ED06F81B413D0CFC140F468
:103AF400D0C141F4450E0401426F530E436F000ED2
:103B0400446FAFEC02F0CFC1D1F3D0C1D2F341EC9A
:103B140012F00101B49FD10ECF6F010ED06FE6EC0D
:103B240016F01AEC12F00101B4A908D0B0C1D1F317
:103B34002EEC12F0E1EC18F000C0B3F1000E01011C
:103B4400631902E1000E6219D8A472D157C226F497
:103B540058C227F48D0E0401286F030E296F81ECDF
:103B640005F08D0E266F030E276F74EC09F0010E1D
:103B7400266F30EC08F000C0B1F101C0B2F100C012
:103B840026F401C027F48D0E0401286F030E296F5B
:103B940081EC05F0670E266F590E276F000E286F13
:103BA40064EC05F08D0E0401266F030E276F74EC90
:103BB40009F0870E266F580E276F000E286F64ECED
:103BC40005F0020E0401266F30EC08F0060E005ECC
:103BD400000E015A00C0AEF101C0AFF100C026F4DE
:103BE40001C027F48D0E0401286F030E296F81ECA8
:103BF40005F08D0E266F030E276F74EC09F089EC27
:103C04000FF000C06CF101C06DF102C06EF103C091
:103C14006FF1DE0E0401266F580E276F000E286F19
:103C240064EC05F06CC10FF46DC110F46EC111F4B5
:103C34006FC112F48D0E0401136F030E146F020E84
:103C4400156F34EC0DF08D0E266F030E276F74EC98
:103C540009F0850E266F590E276F000E286F64EC4D
:103C640005F003018D6B0101B4A945D08D0E04014B
:103C7400406F030E416FD00E426F570E436F000E1C
:103C8400446FAFEC02F0B3C10FF451EC0FF000C07D
:103C940011F401C012F4930E0F6F030E106FFEECBB
:103CA4000CF08D0E266F030E276F74EC09F00301E0
:103CB4008D6B8D0E0401406F030E416FC10E426F78
:103CC400570E436F000E446FAFEC02F0B0C10FF417
:103CD40051EC0FF000C011F401C012F4930E0F6FF9
:103CE400030E106FFEEC0CF08D0E266F030E276F83
:103CF40074EC09F009D00401090E266F580E276FE1
:103D0400000E286F64EC05F07F0E0401266F590E37
:103D1400276F000E286F64EC05F0000E83BE010EC1
:103D24000401406F300E402736EC05F03D0E0401CF
:103D3400266F590E276F000E286F64EC05F0000EF5
:103D440087B6010E0401406F300E402736EC05F0B3
:103D5400360E0401266F590E276F000E286F64EC8F
:103D640005F0000E83B8010E0401406F300E4027A9
:103D740036EC05F02F0E0401266F590E276F000E46
:103D8400286F64EC05F0000E84B8010E0401406F46
:103D9400300E402736EC05F0BA0E0401266F580E9B
:103DA400276F000E286F64EC05F0000E0101B4B516
:103DB400010E0401406F300E402736EC05F04B0E27
:103DC4000401266F590E276F000E286F64EC05F06E
:103DD400000E0101B4BB010E0401406F300E4027F8
:103DE40036EC05F0080E0401266F590E276F000EFD
:103DF400286F64EC05F0000E80B0010E0401406FE2
:103E0400300E402736EC05F0280E0401266F590EBB
:103E1400276F000E286F64EC05F0000E83BC010EC2
:103E24000401406F300E402736EC05F0EAEC05F053
:103E34007AEC11F00101B4BD2ED0B251020802E1B6
:103E4400B15100081DE36CC104F06DC105F06EC1F1
:103E540006F06FC107F0000E006E000E016E700ECA
:103E6400026E830E036EC9EC07F0010ED8B0000E8B
:103E7400006E005205E183AE03D087A601D00AD0BC
:103E84000101000E611902E1000E601903E1B4A5FD
:103E940001D001D011D1010E606F000E616FB4AB7F
:103EA40082D08C9CD10ECF6F010ED06FCFC140F465
:103EB400D0C141F4800E0401426F560E436F000ED0
:103EC400446FAFEC02F0CFC126F4D0C127F474ECF8
:103ED40009F0EAEC05F0010E0401266F000E276FCD
:103EE400010E286F000E296FCFC12AF4D0C12BF424
:103EF40010EC06F05C0E0B6E510E0C6E600E0D6E27
:103F04000D2EFED70C2EFCD70B2EFAD70000B30EC5
:103F1400266F510E276F000E286F64EC05F0570EC4
:103F240004010F6F580E106F000E116F000E010187
:103F3400B4B7010E0401126F75EC0CF07A0E0B6E1F
:103F4400C10E0C6E810E0D6E0D2EFED70C2EFCD7FD
:103F54000B2EFAD700000000220E0401266F500E2B
:103F6400276F000E286F64EC05F0F40E04010F6F48
:103F7400540E106F000E116F000E0101B4B7010E44
:103F84000401126F75EC0CF01F0E0B6E710E0C6EAB
:103F94001E0E0D6E0D2EFED70C2EFCD70B2EFAD74F
:103FA40000000101B49BB4AD53D0B4A951D0D90ED3
:103FB4000401266F510E276F000E286F64EC05F084
:103FC400E1EC18F000C0B3F100C00FF4CFC110F45D
:103FD400D0C111F43BEC0CF0CFC126F4D0C127F4CE
:103FE40074EC09F0EAEC05F0D10E0101CF6F010E7B
:103FF400D06FCFC140F4D0C141F4910E0401426F9F
:10400400560E436F000E446FAFEC02F0B3C10FF4D1
:1040140051EC0FF000C011F401C012F4070E0101BD
:10402400CF2504010F6F000E0101D0210401106F90
:10403400FEEC0CF0020E266F000E276F010E286FA7
:10404400000E296FCFC12AF4D0C12BF410EC06F076
:104054000401F20E266F550E276F000E286F64ECD4
:1040640005F0CFC1D1F3D0C1D2F3D2EC13F000C02C
:1040740068F101C069F100C026F401C027F48D0E77
:10408400286F030E296F81EC05F08D0E266F030E49
:10409400276F74EC09F0EAEC05F0CFC1D1F3D0C17D
:1040A400D2F341EC12F00101B4AD02D0B49DF28818
:1040B4009EEC09F0E6EC16F00001000E6E1902E128
:1040C400010E6D19D8A48BEF24F00101B4BB8BEF62
:1040D40024F05B0E0401266F020E276F7D0E286FFD
:1040E400000E296FE3EC06F000C05BF301C05CF343
:1040F400000E026E0150025C02E100500008D8B0CC
:1041040089EF24F0010E0401266F000E276F70EC76
:1041140006F0010E0401266F000E276F010E286FB2
:10412400000E296F4D0E2A6F560E2B6F000E2C6F4A
:10413400BDEC09F0B40E266F500E276F000E286FE9
:1041440064EC05F04C0E0401266F550E276F000E2B
:10415400286FF3EC05F0D60E0B6E110E0C6EE40E08
:104164000D6E0D2EFED70C2EFCD70B2EFAD70000A9
:104174005B0E0401266F020E276F74EC09F0EAEC63
:1041840005F00201596B5A6B5B0E0401266F020E97
:10419400276F780E286F000E296FE3EC06F0000EEF
:1041A400026E0150025C02E10050000803E20201C9
:1041B400596B5A6B5B0E0401266F020E276F930E28
:1041C400286F000E296FE3EC06F0000E026E01501A
:1041D400025C02E10050000805E2010E0201596F81
:1041E400000E5A6F5B0E0401266F020E276F980EA5
:1041F400286F000E296FE3EC06F000C05BF301C0EA
:104204005CF3000E026E0150025C02E100500008F3
:1042140079E2720E0401406F010E416FA80E426FE5
:10422400520E436F000E446FAFEC02F07B0E04019C
:104234000F6F010E106F040E03015B250401116F53
:10424400000E03015C210401126F0E0E136F000EA9
:10425400146F3DEC0AF0B60E266F550E276F000E54
:10426400286F64EC05F0020E0401266F000E276F20
:1042740070EC06F0010E0401266F000E276F010E8C
:10428400286F000E296F6F0E2A6F560E2B6F000ECB
:104294002C6FBDEC09F0020E266F000E276F010E85
:1042A400286F000E296F720E2A6F010E2B6F10EC0F
:1042B40006F0720E266F010E276F74EC09F0EAEC1B
:1042C40005F09EEC09F0720E04010F6F010E106FE1
:1042D40081EC0AF0B70E0B6EA10E0C6EC30E0D6EC0
:1042E4000D2EFED70C2EFCD70B2EFAD700000000A3
:1042F4005B0E266F020E276F74EC09F0EAEC05F0F2
:104304009EEC09F05B0E0401266F020E276F820EED
:10431400286F000E296FE3EC06F000C05BF301C0C8
:104324005CF3000E026E0150025C02E100500008D2
:10433400D8B0DFD003018D6B630E0401266F580ED5
:10434400276F000E286F64EC05F08D0E04010F6FCB
:10435400030E106F050E03015B250401116F000E9F
:1043640003015C210401126F080E136F000E146F19
:104374003DEC0AF08D0E266F030E276F74EC09F0E6
:104384000101686B696B800E706F000E716F6A6B50
:104394006B6B0201516B526B000E525D02E1080E11
:1043A400515D2FE28D0E5125E96E030E5221EA6E06
:1043B400EE50300A0AE08D0E5125E96E030E5221AB
:1043C400EA6EEE50310A01E003D00101684B692B1B
:1043D4008D0E02015125E96E030E5221EA6EEE5054
:1043E400310A05E1010170516A2771516B23010102
:1043F40071337033719F71BD718F0201514B522B18
:10440400CBD7000E0101691902E1080E681959E1C0
:10441400B4A957D06AC1B0F1240E0401266F580E16
:10442400276F000E286F64EC05F0B0C1D1F32EECB9
:1044340012F0D10E0101CF6F010ED06FCFC140F445
:10444400D0C141F47B0E0401426F580E436F000E3D
:10445400446FAFEC02F0B0C10FF48D0E0401106F85
:10446400030E116F3BEC0CF0CFC10FF4D0C110F46C
:104474008D0E116F030E126F21EC0FF0CFC140F4BB
:10448400D0C141F4E8EC04F000C068F101C069F166
:1044940000500101CF250401406F01500101D021DA
:1044A4000401416FCC0E426F580E436F000E446FEF
:1044B400AFEC02F0CFC1D1F3D0C1D2F341EC12F092
:1044C40016D00101B4A90AD0850E0401266F500E3E
:1044D400276F000E286F64EC05F009D0E80E040184
:1044E400266F520E276F000E286F64EC05F09EECC9
:1044F40009F05B0E0401266F020E276F880E286FE9
:10450400000E296FE3EC06F000C05BF301C05CF31E
:10451400000E026E0150025C02E1005000080DE240
:104524000101B495200E0401266F550E276F000E6D
:10453400286F64EC05F09EEC09F05B0E0401266F15
:10454400020E276F440E286F000E296FE3EC06F06D
:1045540000C05BF301C05CF3000E026E0150025C0C
:1045640002E1005000080DE20101B485640E04016B
:10457400266F540E276F000E286F64EC05F09EEC36
:1045840009F05B0E0401266F020E276F350E286FAB
:10459400000E296FE3EC06F000C05BF301C05CF38E
:1045A400000E026E0150025C02E1005000081BE2A2
:1045B400150E0401266F540E276F000E286F64EC4D
:1045C40005F0CFC1D1F3D0C1D2F3D2EC13F000C0C7
:1045D40068F101C069F1CFC1D1F3D0C1D2F341EC8C
:1045E40012F09EEC09F05B0E0401266F020E276F99
:1045F400520E286F000E296FE3EC06F000C05BF347
:1046040001C05CF3000E026E0150025C02E1005036
:104614000008D8B0BFD0070E03015B25E96E000E79
:104624005C21EA6EEE50310A39E1080E5B25040183
:10463400266F000E03015C210401276F4E0E286FC4
:10464400000E296FE3EC06F000C05BF301C05CF3DD
:10465400000E026E0150025C02E100500008D8A076
:104664008C88080E03015B250401266F000E0301EC
:104674005C210401276F300E286F000E296FE3ECD4
:1046840006F000C05BF301C05CF3000E026E015043
:10469400025C02E100500008D8A08C98070E0301C8
:1046A4005B25E96E000E5C21EA6EEE50320A39E1B8
:1046B400080E5B250401266F000E03015C21040132
:1046C400276F1D0E286F000E296FE3EC06F000C063
:1046D4005BF301C05CF3000E026E0150025C02E168
:1046E40000500008D8A08D88080E03015B25040142
:1046F400266F000E03015C210401276F180E286F3A
:10470400000E296FE3EC06F000C05BF301C05CF31C
:10471400000E026E0150025C02E100500008D8A0B5
:104724008D98F90E0401266F530E276F000E286F23
:1047340064EC05F0CFC140F4D0C141F4970E0401FC
:10474400426F540E436F000E446FAFEC02F00E0E36
:104754000101CF25E16E000ED021E26E006A8CB813
:10476400002A300E002600C0E6FF150ECF25E16EAC
:10477400000ED021E26E006A8DB8002A300E0026A9
:1047840000C0E6FFCFC1D1F3D0C1D2F341EC12F0A7
:104794009EEC09F05B0E0401266F020E276F260EB5
:1047A400286F000E296FE3EC06F000C05BF301C034
:1047B4005CF3000E026E0150025C02E1005000083E
:1047C40043E20101B4BB40D0DE0E0401266F550E56
:1047D400276F000E286F64EC05F0CFC140F4D0C100
:1047E40041F48D0E0401426F550E436F000E446F69
:1047F400AFEC02F0CFC1D1F3D0C1D2F341EC12F04F
:10480400880E0401266F520E276F000E286F64EC89
:1048140005F06F0E04010F6F580E106F000E116F2C
:10482400000E0101B4B7010E0401126F75EC0CF017
:10483400F80E0401266F580E276F000E286F64ECE3
:1048440005F08C8C0101B48B5B0E0401266F020E03
:10485400276F6F0E286F000E296FE3EC06F000C07F
:104864005BF301C05CF3000E026E0150025C02E1D6
:104874000050000823E23B0E0401266F560E276FFA
:10488400000E286F64EC05F0D10E0101CF6F010E0C
:10489400D06FCFC140F4D0C141F4800E0401426F07
:1048A4004D0E436F000E446FAFEC02F0CFC1D1F355
:1048B400D0C1D2F341EC12F09EEC09F00101B4BB7B
:1048C40026D0EF0E0401266F4F0E276F000E286FBF
:1048D40064EC05F0620E04010F6F550E106F000EAC
:1048E400116F000E0101B4B7010E0401126F75ECD3
:1048F4000CF00D0E0B6E2D0E0C6ED70E0D6E0D2ED4
:10490400FED70C2EFCD70B2EFAD7000000009EEC2D
:1049140009F00201574B582B800E006E800E581977
:10492400005C02E157513B0806E20101606B616BD8
:104934000201576B586B000E0001751902E1010E5C
:10494400741963E1EAEC05F0CA0E0401266F000E47
:10495400276F74EC09F0EAEC05F0CA0E0401406F0D
:10496400000E416F5A0E426F000E436F050E446FE6
:1049740005EC05F0000E011802E1000E001805E137
:10498400010E0101626F000E636FCA0E0401406FD5
:10499400000E416F630E426F000E436F060E446FAC
:1049A40005EC05F0000E011802E1000E001803E109
:1049B4000101626B636BCA0E0401406F000E416F0C
:1049C400B60E426F000E436F050E446F05EC05F002
:1049D400000E011802E1000E0018D8B48C8CCA0E27
:1049E4000401406F000E416FC30E426F000E436F0F
:1049F400050E446F05EC05F0000E011802E1000EEF
:104A04000018D8B48C9CE6EC16F0000E6E1902E186
:104A1400020E6D191EE1C00E0401266F530E276F9E
:104A2400000E286F64EC05F021C026F422C027F4A0
:104A34008D0E0401286F030E296F81EC05F08D0E95
:104A4400266F030E276F74EC09F0EAEC05F09EEC78
:104A540009F0000E751902E1020E741924E161C017
:104A640068F162C069F1E6EC16F0680E0401266F85
:104A7400520E276F000E286F64EC05F068C126F40F
:104A840069C127F48D0E0401286F030E296F81EC90
:104A940005F08D0E266F030E276F74EC09F0EAEC17
:104AA40005F0E6EC16F0E6EC16F09EEC09F00101D8
:104AB400B56BB66B0101000E631902E1010E6219B8
:104AC400D8A44DD10A0E046E000E056EB5C100F0D7
:104AD400B6C101F025EC02F008C000F009C001F0F5
:104AE400000E011802E1000E001852E1A20E0401AA
:104AF400266F530E276F000E286F64EC05F0010E2D
:104B04000401266F000E276F70EC06F0070E0B6E83
:104B1400170E0C6E6A0E0D6E0D2EFED70C2EFCD7E2
:104B24000B2EFAD70000010E0401266F000E276F2A
:104B3400010E286F000E296FB30E2A6F560E2B6FCD
:104B4400000E2C6FBDEC09F0020E266F000E276FCD
:104B540070EC06F0070E0B6E170E0C6E6A0E0D6EDF
:104B64000D2EFED70C2EFCD70B2EFAD70000020E0A
:104B74000401266F000E276F010E286F000E296FA7
:104B8400080E2A6F570E2B6F000E2C6FBDEC09F028
:104B94000101B54BB62B7A0E0B6EC10E0C6E810E55
:104BA4000D6E0D2EFED70C2EFCD70B2EFAD700005F
:104BB4000000000E0001751902E1010E7419D8A459
:104BC400CDD0CA0E0401406F000E416F9F0E426F9C
:104BD400000E436F050E446F05EC05F0000E01183E
:104BE40002E1000E001805E1010E0101626F000EE2
:104BF400636FCA0E0401406F000E416FA50E426F31
:104C0400000E436F050E446F05EC05F0000E01180D
:104C140002E1000E001803E10101626B636BDF0E19
:104C24000401266F570E276F000E286F64EC05F001
:104C3400300E010162250401406F36EC05F0090EC7
:104C44000401406F36EC05F0790E0401266F590E0D
:104C5400276F000E286F64EC05F0CA0E0401266F5E
:104C6400000E276F74EC09F0EAEC05F0000E010168
:104C7400631902E1010E62196FE19EEC09F0CA0E9C
:104C840004010F6F000E106F81EC0AF00D0E406FDF
:104C94005DEC05F03D0E0B6EE10E0C6E3F0E0D6EDD
:104CA4000D2EFED70C2EFCD70B2EFAD700000000D9
:104CB4005B0E0401266F020E276F74EC09F0EAEC18
:104CC40005F0010E0401266F000E276F70EC06F04C
:104CD400070E0B6E170E0C6E6A0E0D6E0D2EFED7A0
:104CE4000C2EFCD70B2EFAD70000010E0401266F00
:104CF400000E276F010E286F000E296F190E2A6F00
:104D0400570E2B6F000E2C6FBDEC09F0020E266FB0
:104D1400000E276F70EC06F0070E0B6E170E0C6E6C
:104D24006A0E0D6E0D2EFED70C2EFCD70B2EFAD765
:104D3400000002016B6B020E0401266F000E276F48
:104D4400010E286F000E296F5B0E2A6F020E2B6F67
:104D540010EC06F09EEC09F0E6EC16F0ABD680B051
:104D640002D00101B495000E0301D01902E1000E36
:0C4D7400CF1901E1F8D793EF1DF0FFD735
:10598E0010EE18F0480E006E010E016EF40EF66E5B
:10599E004E0EF76E000EF86EA7EC10F010EE61F0E2
:1059AE00090E006E010E016EC30EF66E580EF76EE6
:1059BE00000EF86EA7EC10F010EE60F0010E006E07
:1059CE00010E016E060EF66E000EF76E000EF86EEC
:1059DE00A7EC10F010EE6AF05F0E006E010E016E75
:1059EE00030EF66E4E0EF76E000EF86EA7EC10F06C
:0259FE00120095
:0100060000F9
:104D80000D0A4364657320646973706F3A0D0A20DD
:104D900044617461204F6E2064656D616E64200D06
:104DA0000A20537572766579204F6E20286F752022
:104DB0004F6666290D0A20536F6D6D65696C0D0A8B
:104DC00020436465204C65643120306E20286F7567
:104DD000204F6666290D0A204D41483D31352F3060
:104DE000392F32392C31363A34353A30302B303491
:104DF0000D0A204D4350313D3030303030303030AE
:034E00000D0A0098
:034E03004F4B0012
:024E06000000AA
:054E080048656C70001C
:024E0D000000A3
:024E0F000000A1
:054E11003437313500CB
:054E1600434D5449006A
:064E1B004D4350313D0043
:0B4E2100537572766579204F666600BD
:054E2C003338333700AC
:054E31004D41483D0069
:024E360000007A
:064E38004465627567008D
:074E3E004E6F726D616C0004
:014E450074F8
:064E46004572726F72005C
:034E4C004F4B00C9
:064E4F004454523D310005
:074E55002B43474D533A00C7
:064E5C004454523D3000F9
:104E62002031384638374A35305F47534D325F5527
:104E7200415254325F55415254315F4C43445F4971
:104E820032435F4D435032333031375F57616B6588
:104E920055705F4F6E4576656E745F775F685F3100
:0A4EA20036303632352E630D0A005B
:104EAC002031384638374A35305F47534D325F55DD
:104EBC00415254325F55415254315F4C43445F4927
:104ECC0032435F4D435032333031375F57616B653E
:104EDC0055705F4F6E4576656E745F323031362E8D
:084EEC006D637070690D0A008E
:054EF400204F6666007E
:044EF900204F6E00D8
:024EFD000000B3
:034EFF004F4B0016
:084F0200536F6D6D65696C00D1
:024F0A000000A5
:054F0C00204F66660065
:0F4F110044617461204F6E2044656D616E6400D1
:0A4F2000537572766579204F6E001C
:044F2A00204F6E00A6
:084F2E00436465204C6564003A
:064F36004465627567008E
:104F3C00205665726966696572206C61207072E931
:104F4C0073656E6365206465207265736973746143
:104F5C006E6365732050756C6C20555020737572A0
:0F4F6C002053434C20657420534441200D0A000C
:104F7B0020496E6974205642524159205541525472
:104F8B00312031393230302C382C4E2C3120657495
:104F9B00205155454354454C2055415254322031F4
:0D4FAB00393230302C382C4E2C310D0A00DC
:104FB800204C69737420616C6C20554E52454144F5
:104FC800206D73672066726F6D20696E626F78203E
:104FD8002841542B434D474C3D52454320554E5292
:074FE800454144290D0A00B8
:104FEF0045666661636520746F7573206C65732009
:104FFF00534D53207265E77573202841542B514D43
:10500F004744413D2244454C20494E424F582229A6
:03501F000D0A0077
:1050220045666661636520746F7573206C657320D5
:10503200534D53207265E77573202841542B514D0F
:105042004744413D2244454C20494E424F58222973
:035052000D0A0044
:10505500205465737420736920656E726567697382
:105065007472E920737572206C65207265736561D1
:1050750075202841542B435245473F31290D0A00DD
:10508500205265667573E965200D0A20504220643B
:105095006520666F726D617420636465203A204DEA
:0F50A5004350313D30303030303030300D0A0064
:1050B4002052656164206D657373616765204E4F8E
:1050C4004E204C5553202841542B434D474C3D22F0
:0F50D40052454320554E5245414422290D0A00B2
:1050E300222B3333363231333334373135220022F6
:1050F3002B333336313431333338333722004E6F69
:0D5103007420617574686F72697A656400CC
:1051100020466169726520526573657420706F75F1
:10512000722072656C616E636572206C65207072AE
:0B5130006F6772616D652E2E0D0A0086
:10513B0020557361676520646520534C45455020AD
:10514B006D6F646520302065742032202C20204345
:0A515B00646520445452200D0A0040
:10516500204E6576657220676F20696E20534C4529
:105175004550206D6F64652841542B5153434C4B6A
:075185003D3029200D0A0056
:10518C00204C656374757265206465206461746578
:10519C00206574206865757265202841542B434343
:0751AC004C4B3F290D0A00E6
:1051B3004E6576657220476F20696E20534C4545D6
:1051C30050206D6F64652841542B5153434C4B3D24
:0651D3003029200D0A0046
:1051D90057616B65557020766961206368616E67F8
:1051E90065206F6E203845204D43503233303137BA
:0451F900203A200038
:1051FD002031657265204C6563747572652041447C
:10520D0043205241312065742041444320524132A4
:04521D00200D0A0056
:105221002031657265204C65637475726520414457
:105231004320524131206574204144432052413280
:04524100200D0A0032
:10524500200D0A436F6E737469747574696F6E20EF
:10525500647520534D5320E020656E766F79657235
:035265000D0A002F
:105268000D0A204465626F7264656D656E74204234
:10527800756666657231205541525431203A2000D6
:10528800476F20696E20534C454550206D6F64650B
:105298002841542B5153434C4B3D3229200D0A00D1
:1052A80041542B43434C4B3D2231352F30392F325B
:1052B800392C31363A34353A30302B3034220D001F
:1052C80020506F776572204F4E206D6F64756C6546
:1052D8002047534D322D636C69636B200D0A200003
:1052E800205265667573E96520636172204D4350ED
:0F52F800323330313720616273656E740D0A00F6
:10530700200D0A20436F6E74656E752064752053F7
:0F5317004D5320E020656E766F7965720D0A00A8
:1053260020313932303020426175642072617465F3
:0F533600204E65676F636520424144200D0A00D9
:105345000D0A496E697420657420316572204465C3
:0F5355006D6172726167652047534D320D0A001A
:1053640020496E6974204D43503233303137203830
:0F5374004520385320656E20493243200D0A0032
:10538300205365742050494E20636F64652841544F
:0F5393002B4350494E3D3132333429200D0A004F
:1053A20020417474656E74652043646520636C618A
:0E53B20076696572205642524159200D0A005C
:1053C000204465626F7264656D656E7420627566F7
:0D53D000666572205541525432200D0A00CE
:1053DD00205072657420706F757220656E766F69DE
:0C53ED00204D736720747874200D0A00B6
:1053F900205265746F75722064276F72647265201C
:0C540900636465204C656473200D0A008C
:105415000D0A456E766F6920446174617320646579
:0B5425006D616E64E96573200D0A00E4
:1054300020546573742070726573656E6365204CCB
:0A544000434420323131390D0A00D7
:10544A0020436F6D706F7365204E756D65726F20A6
:0A545A002841542B434D47533D00F9
:10546400204469616C6F67756520534D53207265E4
:0A5474007461626C6974200D0A0077
:10547E00204572726575722073757220656E766F37
:09548E006920534D53200D0A0062
:105497000D0A5265746F7572204C6564313D20208A
:0854A7004C6564323D200D004C
:1054AF00204E622064652070617320496E697420FC
:0754BF004C4344203D200096
:1054C6002041726D6520525820495420554152544E
:0754D60032202E2E0D0A000A
:1054DD002041726D65205258204954205541525437
:0754ED0031202E2E0D0A00F4
:1054F40041542B514D4744413D2244454C20494E93
:06550400424F58220D0089
:10550A000D0A47534D322050494331384638374AFD
:06551A0035303A0D0A00D5
:105520002053544F50206469616C6F677565205338
:065530004D53200D0A009E
:1055360041542B434D474C3D2252454320554E5234
:06554600454144220D0066
:10554C0041542B434D474C3D2252454320554E521E
:06555C00454144220D0050
:1055620041542B514D4744413D2244454C20494E24
:06557200424F58220D001B
:10557800204E65676F63652062617564207261748F
:0555880065200D0A0082
:10558D000D0A4F4B206D6F6465206D696D696E75E9
:05559D006D20780D00F7
:1055A20020496E69742049324331203130304B68D2
:0455B2007A0D0A0064
:1055B600204D414A206461746520657420486575F4
:0455C60072652000EA
:1055CA0020496E697420446973706C6179204C4378
:0455DA00440D0A0072
:1055DE00204D69736520656E20736F6D6D65696C06
:0455EE00200D0A0082
:1055F20020436F6D706F7365204D7367206C656E0D
:035602003D200048
:10560500204E65676F636520726575737369200D3C
:025615000A0089
:10561700204572723A204E6F204D4350323330315D
:0256270037004A
:10562900205068617365206427696E697420656E0E
:0256390020004F
:10563B002048656C702064656D616E64E965200DB2
:02564B000A0053
:10564D00526563657074696F6E20534D5320202031
:01565D00004C
:10565E0020496E74727573696F6E204541313D201D
:01566E00003B
:10566F004D414A206461746520686575726520201C
:01567F00002A
:1056800052657665696C2047534D32202F44545241
:015690000019
:105691003820496E703D202020202020202020200D
:0156A1000008
:1056A2005068617365206427696E697420656E2095
:0156B20000F7
:1056B300546573742047534D322D636C69636B20BB
:0156C30000E6
:1056C40053746570203A202E2E2E2E2E2F20352036
:0156D40000D5
:1056D500202020202020706173202F2035202020BD
:0156E50000C4
:1056E600496E69742047534D322D436C69636B20B4
:0156F60000B3
:1056F7004E65676F636520626175642072617465CA
:0157070000A1
:105708006176656320514E4156494741544F5220B6
:015718000090
:10571900436465202047534D322D636C69636B20C8
:01572900007F
:10572A0041647265737365204F4B203078343020A2
:01573A00006E
:10573B00696E69204D435032333031372049324343
:01574B00005D
:10574C0042414420416472657373203078343020B8
:01575C00004C
:10575D0020526573657420436C69636B65723220EA
:01576D00003B
:10576E0042414420496E6974205374657020202094
:01577E00002A
:10577F00436F6D706F7365204E756D65726F20206E
:01578F000019
:1057900053543D20202044493D2020534F3D20209C
:0157A0000008
:1057A100436865636B20446576696365204020002A
:1057B10020456E766F6920534D53204F4B203A00A0
:0F57C1003B2038533D2030303030303030300016
:0F57D0003B2038453D2030303030303030300015
:0E57DF00204D6F6465204465627567203D00B3
:0E57ED00206973206E6F7420666F756E640005
:0E57FB0041542B4350494E3D313233340D00A2
:0E5809003B204E6F204D43503233303137007C
:0D58170038453D203030303030303030002A
:0D58240020416363657074E965200D0A0082
:0D58310038533D2030303030303030300002
:0D583E002041444320496E6974200D0A008A
:0C584B0041542B5153434C4B3D300D0099
:0C58570041542B5153434C4B3D300D008D
:0C586300436465204D435031203A200082
:0C586F0041542B5153434C4B3D320D0073
:0C587B0020436465204D435031203D0067
:0B5887003B20454132204E6F773D0072
:0A5892000D0A20456E642E0D0A0079
:0A589C0020666F756E64204F4B000C
:0A58A60041542B435245473F0D00CB
:0A58B00041542B43434C4B3F0D00C5
:0958BA003B4469616C6F673D001D
:0258C3000000E3
:0758C5004E6F726D616C0073
:0958CC00202E2E4F4B200D0A0086
:0958D50020464F5343203D200002
:0958DE003B54656D70463D20004D
:0958E70041542B434D47533D0091
:0858F000204C4432203D200051
:0858F8004454523D310D0A0039
:08590000204C4431203D200041
:085908003B20535441543D00C3
:085910002054656D703D20007C
:0859180020425031203D200027
:0859200020425032203D20001E
:075928003B204454523D00F6
:07592F003B204C44323D0017
:075936003B204C44313D0011
:07593D003B204250323D0007
:0759440054656D703D200069
:07594B003B20534F4D3D00CE
:075952002E2E42414421000A
:07595900207061732F35007F
:0759600020537465703A004A
:06596700204541313D0026
:06596D004541313D200020
:065973002E2E204F4B0018
:06597900204364653D00BF
:06597F003B4250313D00E7
:055985006465672000CD
:04598A0041540D0077
:020000040001F9
:06FFF800ACF705FFF0FF6D
:00000001FF
